:1000000000308A00D0290000831A0A289100030ECC
:1000100092000F2883129100030E920092140A0896
:1000200099008A018313910E040893000C08940030
:100030000D0895000E0896000F089700100898000C
:1000400083128B1E25280B19852813088400140899
:100050008C0015088D0016088E0017088F001808F0
:10006000900019088A00120E83008312110E921854
:10007000831609008D018E018C018F012A08031D52
:100080004428290803195E281030AB000310A70D7F
:10009000A80D8C0D8F0D2A080F02031D5128290869
:1000A0000C02031C5A2829088C02031C8F032A08FF
:1000B0008F0203148D0D8E0DAB0B4628000000340B
:1000C0008C018D012508031026188C078C0C8D0CD3
:1000D000A6188C078C0C8D0C26198C078C0C8D0C9B
:1000E000A6198C078C0C8D0C261A8C078C0C8D0C89
:1000F000A61A8C078C0C8D0C261B8C078C0C8D0C77
:10010000A61B8C078C0C8D0C003463308100A1037E
:100110001C08A8001B08A700AA016430A9003A2007
:100120000D089D001C08A8001B08A700AA010A30A2
:10013000A9003A200E08A6000D08A5000E08A80088
:100140000D08A700AA010A30A9003A200C089E0059
:100150001C08A8001B08A700AA010A30A9003A2021
:100160000C089F00200BC728A00A831606108312D4
:100170000610831606118312061522081D04A50019
:10018000003083168500831225088500F528200895
:10019000023C031DDE28A00A8316061183120611F5
:1001A000831686108312861422081E04A5000030D0
:1001B00083168500831225088500F5282008033C56
:1001C000031DF5280130A0008316861083128610C7
:1001D000831606108312061422081F04A50000309F
:1001E000831685008312250885002108643C0319C5
:1001F000FC28A108031D8D29831686168312861AF2
:1002000014299B0A03199C0A1C08023C0318132991
:10021000FF3A031D0F291B08E73C0318132903307D
:100220009C00E7309B008D29831606168312061A60
:100230002E299B08031D22299C08031D22299B0AA5
:1002400003199C0A1B0803199C039B0B2D299C086E
:10025000031D2D299C0101309B008D2983168615D5
:10026000831286198D29A208031D88299B08031D66
:100270003C299C0803198829831686138312861744
:100280001030A2000B3089001D0888000B088C007C
:100290008B130B088D008316081555308900AA3082
:1002A0008900881488185229081183120D088C1BA4
:1002B0008B000C3089001E0888000B088C008B1303
:1002C0000B088D008316081555308900AA30890067
:1002D000881488186929081183120D088C1B8B005B
:1002E0000D3089001F0888000B088C008B130B0849
:1002F0008D008316081555308900AA3089008814AE
:1003000088188029081183120D088C1B8B008D29F9
:100310008316861383128613A201A108031DCD291B
:100320002208103C031DCD291B0803199C039B0BBD
:10033000CB299C08031DCB298316861383128613B1
:10034000A2010B30890083160814831208089D004F
:100350000C30890083160814831208089E000D30A3
:10036000890083160814831208089F009C011F0847
:100370009B001E08A5000A30A60060200D089B0700
:1003800003189C0A1D08A5006430A60060200D0813
:100390009B0703189C0AC830A1000B118A1125285D
:1003A00084011F3083050130A000C830A100A201E4
:1003B000831681170108C039043881000B3083127D
:1003C000890083160814831208089D000C308900E8
:1003D00083160814831208089E000D3089008316C6
:1003E0000814831208089F009C011F089B009A01B3
:1003F0008B1B9A178B131E08A5000A30A6006020DD
:100400009A1B8B170D089B0703189C0A9A018B1BDC
:100410009A178B131D08A5006430A60060209A1B54
:100420008B170D089B0703189C0A8B168B17172A2E
:02043000630067
:02400E00F93F78
:00000001FF
